:020000040000FA
:2B000000FFFF62FF2500FFFFFFFFFFFFFFFFFFFFFFFFFFFFFFFFFFFFFFFFFFFFFFFFFFFFFFFFFFFFFFFFFFFFFFFFFF76
:2B002B006071DDC17517D71DDCC57587C57587C55DDC050000000018DCC575DD6159DCC57507771916D71D966501E5FD
:2B005600E0280AA1288EA2108AA32884A32884A3388A0300000000108AA3280AE1388AA32884E2108EA2108EE380EC64
:2B008100000000000000000000000000000000000000000000000000000000000000000000000000000000000080E7ED
:2B00AC00000000000000000000000000000000000000000000000000000000000000000000000000000000000080E7C2
:2B00D700800000000028000000020000020000022001120000000000000A00008020200200008000080000088A80EFC8
:2B010200600000000000000000040090000090000000000000000000000000000001000200002440020000420081E33F
:2B012D000000000000000000000000000000000000000000000000000000000000000000000000000000000000A0C542
:2B015800100008000000000000000000000000000000000000000000000000000000000000000000000000000000FF65
:2B018300000040000000000000000000000000000000000000000080000000000000000000000000000000000000A3EE
:2B01AE000C0040000000000000000000000000000000000000000000000000000000000000000000000400000090FA4C
:2B01D900000000000000000000000000000000000000000000000000000000000000000000000000000000000080E794
:2B020400000000000000000000000000000000000000000000000000000000000000000000000000000000000008EFD8
:2B022F00000000000000000000000000000000000000000000000000000000000000000000000000000000000080E73D
:2B025A00000000000000000000000000000000000000000000000000000000000000000000000000000000000080E712
:2B028500000000000001000000000000000000000000000000000000000000000000000000000000000000000080F7D6
:2B02B000100000100000000000000000000000000010000000000000000000000000000000000000000000000080F67D
:2B02DB00000000000000000000000000000000000000000000000000000000000000000000000000000000000080E791
:2B030600000000000000000000000000000000000000000000000000000000000000000000000000000000000008EFD5
:2B033100000000000000000000000000000000000000000000000000000000000000000000000000000000000080E73A
:2B035C00000110000100000000000010000100000040000000000040000440000400000440000400001000000480B3FC
:2B038700000280000880000002200000000000200000080000000080000000002000000000800100800000000080FED8
:2B03B200820000000000000002200000000000200000000000000000000000000000000000800000800000000000CD8F
:2B03DD00024000000000000000000000000000000000000000000000000000000000000000000000000000000008E9C2
:2B040800040000000880000000000000000000000000000000000000000000000000000000000000000000000008EB4A
:2B0433008243800000000000000000000000000000000800000000C000000000A000000000000300000000000088A7BF
:2B045E00020000000000000000000000000000000000000000000000000000000000000000000000000000000008ED7C
:2B048900020000000000000000000000000000000000000000000000000000000000000000000000000000000080E5E1
:2B04B400800008800008800008800008800008800008000000000020000220000220000220000220000220000280E7BA
:2B04DF00800008800008800008800008800008800008000000000020000220000220000220000220000220000280E78F
:2B050A00000000000000000000000000000000000000000000000000000000000000000000000000000000000080E75F
:2B0535000200180000000000000000000000000000180000000000000000000000000000600000000000000000088B76
:2B056000020002000000000000000000000000000002000000000000000000000000000008000000000000000088E5F5
:2B058B0004001C00000000000000000000000000001C0000000000000000000000000000700000000000000000908584
:2B05B600020002000000000000000000000000000002010000000000000000000000000008100000000000000088F47F
:2B05E10002003A02000000000000000000000000001A0000000000000000000000000000E8000000000000000008A304
:2B060C00020000010000000000000000000000000000020000000000000000000000000000040000000000000008EAC8
:2B063700000018000000000000000000000000000038000000000000000000000000000060000000000000000080A3C5
:2B066200000000000000000000000000000000000000000000000000000000000000000000000000000000000080E706
:2B068D00000018000000000000000000000000000000000000000000000000000000000000000000000000000000FE2C
:2B06B800020002000000000000000000000000000000000000000000000000000000000000000000000000000008CD3E
:2B06E30002001C000000000000000000000000000000000000000000000000000000000000000000000000000088B492
:2B070E00040022000000000000000000000000000000000000000000000000000000000000000000000000000090F01A
:2B07390002001A000000000000000000000000000000000000000000000000000000000000000000000000000088D41D
:2B076400020000010000000000000000000000000000000000000000000000000000000000000000000000000008EC73
:2B078F00020018000000000000000000000000000000000000000000000000000000000000000000000000000088F4A9
:2B07BA00000000000000000000000000000000000000000000000000000000000000000000000000000000000080E7AD
:2B07E500000018000000000000000000000000000000000000000000000660000000000000000000000000000000FE6D
:2B081000000002000000000000000000000000000000000000000000800008000000000000000000000000000080C7EC
:2B083B0000001C000000000000000000000000000000000000000000000770000000000000000000000000000088B6C1
:2B08660002000200000000000000000000000000000000000000000080000A200000000000000000000000000008CDE4
:2B08910002001A010000000000000000000000000000000000000000800E68000000000000000000000000000090CCCD
:2B08BC00020000010000000000000000000000000000000000000000004000040000000000000000000000000008ECD6
:2B08E700020018000000000000000000000000000000000000000000000660000000000000000000000000000088F4EA
:2B091200000000000000000000000000000000000000000000000000000000000000000000000000000000000008EFC3
:2B093D00000018000000000000000000000000000000000000000000000000000000000000000000000000000000FE79
:2B096800000002000000000000000000000000000000000000000000000000000000000000000000000000000080C71B
:2B09930000001C000000000000000000000000000000000000000000000000000000000000000000000000000000BE5F
:2B09BE00020002010000000000000000000000000000000000000000000000000000000000000000000000000080C4C5
:2B09E90002003A000000000000000000000000000000000000000000000000000000000000000000000000000088F629
:2B0A1400040000010000000000000000000000000000000000000000000000000000000000000000000000000008EAC0
:2B0A3F00020018000000000000000000000000000000000000000000000000000000000000000000000000000088F4F6
:2B0A6A00020000000000000000000000000000000000000000000000000000000000000000000000000000000008ED6A
:2B0A95000200180000000000000000008001000000000000000000000000000000000000000000000000000006808392
:2B0AC000000002000000000000000000200000000000000000000000000000000000000000000000000000800000EF7A
:2B0AEB0000001C000000000000000000C0010000000000000000000000000000000000000000000000000000078090EC
:2B0B1600000002100000000000000000201000000000000000000000000000000000000000000000000000800880FE6C
:2B0B410000001A000000000000000000A00300000000000000000000000000000000000000000000000000800E08A393
:2B0B6C00020000010000000000000000001000000000000000000000000000000000000000000000000000004008E91A
:2B0B97000200180000000000000000008001000000000000000000000000000000000000000000000000000006909270
:2B0BC200020000000000000000000000000000000000000000000000000000000000000000000000000000000008ED11
:2B0BED00020018000000000000000000000000000000000000000000000000000000000000000000000000000088F447
:2B0C1800000002000000000000000000000000000000000000000000000000000000000000000000000000000008CFD8
:2B0C430000001C000000000000000000000000000000000000000000000000000000000000000000000000000000BEAC
:2B0C6E00000002080000000000000000000000000000000000000000000000000000000000000000000000000080CF02
:2B0C990000001A000000000000000000000000000000000000000000000000000000000000000000000000000000DE38
:2B0CC400020000010000000000000000000000000000000000000000000000000000000000000000000000000008EC0E
:2B0CEF00020018000000000000000000000000000000000000000000000000000000000000000000000000000088F444
:2B0D1A00040000000000000000000000000000000000000000000000000000000000000000000000000000000090F228
:2B0D4500820100000000000000000000000000000000000000000060000000000600000600000000000600000088F412
:2B0D7000220000000000000000000000000000000000000000000008000000800000800000000000800000000008CDD9
:2B0D9B00C20100000000000000000000000000000000000000000070000000000700000700000000000700000088B4A9
:2B0DC600200000000000000000000000000000000000000000000008000000800004800800000000804000000000838B
:2B0DF100A01300000000000000000000000000000000000000000068080000800E00800600000000800600000080F5A5
:2B0E1C00001000000000000000000000000000000000000000000000040000004000004000000000008000000080EA2D
:2B0E4700800100000000000000000000000000000000000000000060000000000600000600000000000E00000080FE07
:2B0E7200020000000000000000000000000000000000000000000000000000000000000000000000000000000008ED5E
:2B0E9D000200188001000000000000180000000000000000000000000000000000000000000006000000000000889257
:2B0EC800020002200000000000000002000000000000000000000000000000000000000000800000000000000088C50C
:2B0EF30002001CC0010000000000001C000000000000000000000000000000000000000000000700000000000088C387
:2B0F1E00000002220000000000000002080000000000000000000000000000000000000000800000000000000000C535
:2B0F490000003AA0010100000000003A000000000000000000000000000000000000000000800604000000000080E07D
:2B0F7400000000011000000000000000010000000000000000000000000000000000000000004000000000000080E29E
:2B0F9F00020018800100000000000018000000000000000000000000000000000000000000000600000000000040DE50
:2B0FCA008A00088000000000000000088000000000080000000000200002200002000002200002000002000002C08BA3
:2B0FF500000000000000000000000000000000000000000000000000000000000000000000000000000000000080E76A
:2B102000000000000008800008800000000008800000000000000000000000000020000000000020000020000080C568
:2B104B00400004400008800008800004400008800004000000000010000110000120000110000120000120000180D42C
:2B10760000040010000000000000000000000800000000000000000000A000001000000000000040000000100000E44F
:2B10A100000000000000000000000000000000000000000000000000000000000000000400000040000000000080E779
:2B10CC00000000000002000002000000200000000000000000000000000000000010000000000000800008100080C6E7
:2B10F700000000020000000000000000000080000000000000000000000000000000000000000000000000000000E567
:2B112200000408900002000002000008200088000000000000000000002000001010000400000240800008000000A3A1
:2B114D00800010000000000000000000000000000000000000000000000000000000000000000000000000000000FEE9
:2B117800000000000000000000000000800000000000000000000000000000000002000000000000000000000100DEEB
:2B11A300000000000000000000000000000000000000000000000000000000000000000100000004000000000080B6E6
:2B11CE00000000000000000000000000000000000000000000000000000001000000000000000000000000000080F77E
:2B11F9000000000000000000000000000000000000000000000000000000000000000000000000000000000000B0D447
:2B122400000000020000000000000000040000000000000000000000000000080000000000000000000000000080E928
:2B124F00100000000000000000000000000000000000000000000000000000000000000000000000000000000080F7ED
:2B127A00000000000000000000000000000000000000000000000000000000000000000000000000000000000080E7E2
:2B12A500000000000000000000000000000000000000000000000000000000000000000000000000000000000080E7B7
:2B12D000000000000000000000000000000000000000000000000000000000000000000000000000000000000080E78C
:2B12FB00040004000000000000000000000000000000000000000000000000000000000000000000000000000080A39D
:2B132600000000000000000000000000000000000000000000000000000000000000000000000000000000000080E735
:2B1351000000000000000000000000000000000000000000000000000000000000000000000000000000000000A0C50C
:2B137C00000000000000000000000000000000000000000000000000000000000000000000020000000000000090F4C0
:2B13A700000000000000000000000000000000000000000000000000000000000000000000000000000000000080E7B4
:2B13D200100000000000000000000000000000000000000000000000000000000000000000000000000000000008FFD9
:2B13FD00000000000000000000000000000000000000000000000000000000000000000000000000000000000080E75E
:2B142800020000000000000000000000000000000080000000000000001000000000000000000000000000000000E423
:2B145300000000000000000000000000000000000000000000000000000000000000000000000000000000000080E707
:2B147E00000000000000000000000000000000000000000000000000000000000000000000000000000000000080E7DC
:2B14A9000000000000000000000000000000000000000000000000000000000000000000000000000000000000C0A3B5
:2B14D400000000000000000000000000000000000000000000000000000000000000000000000000000000000080E786
:2B14FF00000000000000000000000000100000000000000000000000000000000000000000000040000000000080B33F
:2B152A00100000000040000000000000000000000000000000000000000000000000000000000000000000010008BA83
:2B155500000000000000000000000000000000000000000000000000000000000000000000000000000000000080E704
:2B158000000000000000000000000000000000000000000000000000000000000000000000000000000000000080E7D9
:2B15AB00000000000000000000000000000000000000000000000000000000000000000040000000000000000080A3B2
:2B15D600000010000010000140000110000010000010000000000040000440000440000440000440000440000480B28E
:2B160100000000200000200002000000000800000000080000000000022000220000000000000000802000000080E721
:2B162C00020000200000200000000000000000000000000000000000000000000000000000000000000000000008ED5C
:2B165700020000000000000000000000000000000000000000000000000000000000000000000000000000000008ED71
:2B168200040000000000000000000000000800000000000000000000022000020000000000000000002000000010F2EB
:2B16AD00020000000000000002000000000000000000080000000000000000200000000000000000800000000088EDF1
:2B16D800020000000000000000000000000000000000000000000000000000000000000000000000000000000008EDF0
:2B170300020000000000000000000000000000000000000000000000000000000000000000000000000000000008EDC4
:2B172E00800008800008800008800008800008800008000000000020000220000220000220000220000220000280E72D
:2B175900800008800008800008800008800008800008000000000020000220000220000220000220000220000280E702
:2B178400000000000000000000000000000000000000000000000000000000000000000000000000000000000080E7D3
:2B17AF0000000000000000000000000000000000001800000000000000006000000000000000000000000000000098FF
:2B17DA00020000000000000000000000000000000002000000000000000008000000000000000000000000000088C58B
:2B18050002000000000000000000000000000000001C000000000000000070000000000000000000000000000088C3DF
:2B183000020000000000000000000000000000000002040000000000000008000000000000000000000000000088C134
:2B185B0002000000000000000000000000000000003A0000000000000000E8200000000000000000000000000088B8DE
:2B188600000000000000000000000000000000000000010000000000000000040000000000000000000000000080E2D0
:2B18B10000000000000000000000000000000000001800000000000000006000000000000000000000000000000098FC
:2B18DC00000000000000000000000000000000000000000000000000000000000000000000000000000000000080E77A
:2B190700000000000000000000000000000000000000000000000000000000000000000000000000000000000080E74E
:2B193200000000000000000000000000000000000000000000000000000000000000000000000000000000000080E723
:2B195D00020000000000000000000000000000000000000000000000000000000000000000000000000000000008ED68
:2B198800020000000000000000000000000000000000000000000000000000000000000000000000000000000008ED3D
:2B19B300020000000000000000000000000000000000000000000000000000000000000000000000000000000008ED12
:2B19DE00020000000000000000000000000000000000000000000000000000000000000000000000000000000008EDE7
:2B1A0900000000000000000000000000000000000000000000000000000000000000000000000000000000000080E74B
:2B1A3400000000000000000000000000000000000000000000000000000000000000000000000000000000000080E720
:2B1A5F00000000000000000000000000000000000000000000000000000000000000000000000000000000000080E7F5
:2B1A8A00000000000000000000000000000000000000000000000000000000000000000000000000000000000080E7CA
:2B1AB500020000000000000000000000000000000000000000000000000000000000000000000000000000000008ED0F
:2B1AE000020000000000000000000000000000000000000000000000000000000000000000000000000000000008EDE4
:2B1B0B00040000000000000000000000000000000000000000000000000000000000000000000000000000000090F229
:2B1B3600020000000000000000000000000000000000000000000000000000000000000000000000000000000008ED8D
:2B1B6100020000000000000000000000000000000000000000000000000000000000000000000000000000000008ED62
:2B1B8C00020000000000000000000000000000000000000000000000000000000000000000000000000000000008ED37
:2B1BB700000000000000000018000000000000000000000000000000000000000000000000000000000600000000984D
:2B1BE200000000000000000002000000000000000000000000000000000000000000000000000000800000000000CF87
:2B1C0D0000000000000000001C000000000000000000000000000000000000000000000000000000000700000000C9C0
:2B1C3800020000000000000002010000000000000000000000000000000000000000000000000000800800000080CCA8
:2B1C630002000000000000001A000000000000000000000000000000000000000000000000000000800600000008BAF2
:2B1C8E00040000000000000000020000000000000000000000000000000000000000000000000000004000000008EDF0
:2B1CB900020000000000000038000000000000000000000000000000000000000000000000000000000600000088B088
:2B1CE400020000000000000000000000000000000000000000000000000000000000000000000000000000000008EDDE
:2B1D0F000200000000000000000000000000180000000000000000000000000000000006000000000000000000009AEF
:2B1D3A00000000000000000000000000000002000000000000000000000000000000800000000000000000000000CF2D
:2B1D650000000000000000000000000000001C000000000000000000000000000000000700000000000000000000C967
:2B1D9000000000000000000000000000000002100000000000000000000000000000800000000000000000000000DFB7
:2B1DBB0002000000000000000000000000003A000000000000000000000000000000804E000000000000000000889CCF
:2B1DE600020000000000000000000000000000010000000000000000000000000000004000000000000000000008E89F
:2B1E11000400000000000000000000000000180000000000000000000000000000000006000000000000000000108DE7
:2B1E3C00020000000000000000000000000000000000000000000000000000000000000000000000000000000008ED84
:2B1E6700020000000000000000000018000000000000000000000000000000000000000000000000000000000088F4BA
:2B1E9200020000000000000000000002000000000000000000000000000000000000000000000000000000000008CD4C
:2B1EBD0000000000000000000000001C000000000000000000000000000000000000000000000000000000000000BE20
:2B1EE800000000000000000000000002000000000000000000000000000000000000000000000000000000000080C786
:2B1F130000000000000000000000001A100000000000000000000000000000000000000000000000000000000000CEAB
:2B1F3E00000000000000000000000000010000000000000000000000000000000000000000000000000000000008EE81
:2B1F6900020000000000000000000018000000000000000000000000000000000000000000000000000000000088F4B7
:2B1F9400020000000000000000000000000000000000000000000000000000000000000000000000000000000090F49C
:2B1FBF00020000000018800100800100000000000000000000000060000600000660000060000000000060000688922F
:2B1FEA00020000000002200000200000000000000000000000000008800000800008000008000000000008800088C59B
:2B20150000000000001CC00100C00100000000000000000000000070000700000770000070000000000070000788C1E4
:2B20400000000000000222800020020000000000000000000000000880800080000A100008000000000008880000D79E
:2B206B0000000000003AA00100A00100000000000000000000000068C00E00800EE80000680400000000E8800E0496A6
:2B209600000000000000011000001000000000000000000000000000044000004000040000040000000000044080E2CC
:2B20C100020000000018800100800100000000000000000000000060000600000660000060000000000060000688922C
:2B20EC00020000000000000000000000000000000000000000000000000000000000000000000000000000000008EDD2
:2B211700040018000000000000000000000000000000000000000000000000000000000000000660000000000010EB20
:2B214200020002000000000000000000000000000000000000000000000000000000000000800008000000000008CD11
:2B216D0002001C000000000000000000000000000000000000000000000000000000000000000770000000000088B476
:2B219800020002000000000000000000000000000000000000000000000000000000000000800008000000000008CDBB
:2B21C30000003A080000000000000000000000000000000000000000000000000000000000808668040000000000F845
:2B21EE00000000010000000000000000000000000000000000000000000000000000000000004000040000000080E61B
:2B2219000C0018000000000000000000000000000000000000000000000000000000000000000660000000000030C11F
:2B2244000400080000088000088000080000080000080000000000200002200002200002200002200002200002C0A708
:2B226F00000000000000000000000000000000000000000000000000000000000000000000000000000000000080E7DD
:2B229A00800000800000000000000000800000800000000000000000000000000000000000000000000000000080E7B2
:2B22C500800004800004400004400004800004800004000000000010000110000110000110000110000110000180E789
:2B22F00000000200000000000000280000000008000000000000000000A040000000100000810000000000008080928E
:2B231B00000000000000000000000000000000000000000000000000000000000000000000000000000000000080E730
:2B234600000000000010000100000100000002000000000000000008000440000040100000000000000000000400CEEA
:2B237100001000000000000000000000000000000080000000000000024000000000000000000000000000028000EA03
:2B239C00001002000000000000000800000002080080000000000008026000000000000000810020000000020080CB1A
:2B23C700000000000000000000000000000000000000000000000000000000000000000000000800000000000000E7FC
:2B23F200000000000000000010000000000000000000000000000000000000000000000000000000000000000080F63A
:2B241D00000000000000000000400000000000000000000000000000000000000000000200000000000000000080854D
:2B244800000000000000000000000000000000000000000000000000000000000001000000000000000000000080F7F1
:2B247300120000000000000000000000000000000000000000000000000000100000000000000000000100000028DE15
:2B249E00080000000000002000000000000000000000000000000000000000000000000000000000000000000080ED7E
:2B24C900000000000000000000000000000000000000000000000000000000000000000000000000000000000080E781
:2B24F400000000000000000000000000000000000000000000000000000000000000000000000000000000000080E756
:2B251F00000000040000000000000000000000000000000000000000400000000000000000000000000000000080A32A
:2B254A00000000000000000000000000000000000000000000000000000000000000000000000000000000000080E7FF
:2B257500000000000000000000000000000000000000000000000000000000000000000000000000000000000082C7F2
:2B25A000000000000000000000000000000000080000000000000000000000000000000000000000000000000080EF99
:2B25CB00120000000000000000000000000000000000000000000000000000000000000000000000000000000038CECD
:2B25F600000000000000000000000000000000000000000000000000000000000000020000000000000000000080E553
:2B262100040000000000000000000000000000000000000000000000000000000000000000000000000000000090F208
:2B264C00000000000000000000000000000000000000000000000000000000000000000000000000000000000008EF6C
:2B267700000000000000000000000000000000000400000000000000000000000000000000000000000000000080A311
:2B26A200000000000000000000000000000000000900000000000000000000002000000000000000000000000020D6EE
:2B26CD00080000000000000000000000000000000000000000000000000000000000000000000000000000000080EF6B
:2B26F800000000000000000000000000000000000000000000000000000000000000000000000000000000000080E750
:2B272300100000000000000000000000000000000000000000000000000000000000000000000000000000000080F704
:2B274E00000000000000000000000000000000000000000000000000000000000000000000000000000000000080E7F9
:2B277900000000000000000000000000000000000000000000000000000000000000000000000000000000000800E746
:2B27A4000C0000000000000000000000000000000000000000000000000000000000000420000000000000000008854D
:2B27CF00000000000000000000000000000000000000000000000000000000000000000000000000000000000080E778
:2B27FA00000000000000000000000000000000000000000000000000000000000000000000000000000000000080E74D
:2B282500000000000000000100000000000000000000000000000000000000000000000000000000000000000080F611
:2B285000000000000100000100400100000100000410000000000040000040000440001040000440000440000480F3F2
:2B287B000008020080000000000010002000000000C200000000000000000880000002200800200000080000008080DC
:2B28A600020002000000000000000000200000000002000000000000000008000000000008000000000000000080C58C
:2B28D100020000000000000000000000000000004000040000000000000000000000000000000000000000000008EDA1
:2B28FC00040800000000000000001000000000000000000000000000000000000000022000000000000000000088EA01
:2B2927000200000080000000000000000000000000D004000000000000000080000000000000A000000C00000088F289
:2B295200020000000000000000000000000000000000000000000000000000000000000000000000000000000008ED63
:2B297D00020000000000000000000000000000000000000000000000000000000000000000000000000000000080E5C8
:2B29A800800008800008800008800008800008800008000000000020000220000220000220000220000220000280E7A1
:2B29D300800008800008800008800008800008800008000000000020000220000220000220000220000220000280E776
:2B29FE00000000000000000000000000000000000000000000000000000000000000000000000000000000000080E747
:2B2A2900020000800100000000000000000000800100000000000000000000000000000000000000000000000008ED89
:2B2A5400020000200000000000000000000000200000000000000000000000000000000000000000000000000008ED20
:2B2A7F00040000C00100000000000000000000C00100000000000000000000000000000000000000000000000090F224
:2B2AAA00020000200200000000000000000000201000000000000000000000000000000000000000000000000008CED7
:2B2AD500020000A00100000000000000000000A00100000000000000000000000000000000000000000000000008ED9D
:2B2B0000020000001000000000000000000000002000000000000000000000000000000000000000000000000008EE82
:2B2B2B00000000800100000000000000000000800300000000000000000000000000000000000000000000000080C536
:2B2B5600000000000000000000000000000000000000000000000000000000000000000000000000000000000080E7ED
:2B2B8100000000000000000000000000000000800118000000000000000000000000000000000000000000000080E729
:2B2BAC00020000000000000000000000000000200002000000000000000000000000000000000000000000000008EDE5
:2B2BD700020000000000000000000000000000C0011C000000000000000000000000000000000000000000000008EDFF
:2B2C0200040000000000000000000000000000200002010000000000000000000000000000000000000000000090F3FD
:2B2C2D00020000000000000000000000000000A0233A000000000000000000000000000000000000000000000008EF86
:2B2C5800020000000000000000000000000000002000010000000000000000000000000000000000000000000008EE38
:2B2C8300020000000000000000000000000000800318000000000000000000000000000000000000000000000008CFB2
:2B2CAE00000000000000000000000000000000000000000000000000000000000000000000000000000000000080E794
:2B2CD900000000000000000000000000000000000000000000000000000000000000000060000000000000000080816F
:2B2D0400000000000000000000000000000000000000000000000000000000000000000008000000000000000000EFAD
:2B2D2F000000000000000000000000000000000000000000000000000000000000000000700000000000000000089869
:2B2D5A00020000000000000000000000000000000000000000000000000000000000000008040000000000000088E1D7
:2B2D85000200000000000000000000000000000000000000000000000000000000000000E80000000000000000909A0F
:2B2DB000020000000000000000000000000000000000000000000000000000000000000000040000000000000008E901
:2B2DDB000200000000000000000000000000000000000000000000000000000000000000600000000000000000088BD8
:2B2E0600000000000000000000000000000000000000000000000000000000000000000000000000000000000008EFAA
:2B2E3100000000000000000000000000000000800100000000000000000000000600000000000060000000000000FE91
:2B2E5C00000000000000000000000000000000200000000000000000000000800000000000000008000000000080C75C
:2B2E8700000000000000000000000000000000C00100000000000000000000000700000000000070000000000000BE2A
:2B2EB200020000000000000000000000000000200001000000000000000000800001000000000008200000000008ED34
:2B2EDD00020000000000000000000000000000A00100000000000000000000800E000000000000E8000000000088D455
:2B2F0800040000000000000000000000000000002000000000000000000000004000000000000000040000000090F0B6
:2B2F3300020000000000000000000000000000800300000000000000000000000600000000000060000000000088D62A
:2B2F5E00020000000000000000000000000000000000000000000000000000000000000000000000000000000008ED51
:2B2F8900020000000000000000000000000000800100000000000060000000000000000000000000000000000688F4B8
:2B2FB400000000000000000000000000000000200000000000000008000000000000000000000000000000800080C703
:2B2FDF00000000000000000000000000000000C00100000000000070000000000000000000000000000000000700BED1
:2B300A00000000000000000000000000000000204000000000000008000000000000000000000000000000800080C370
:2B303500000000000000000000000000000000A00300000000000068400000000000000000000000000000808600B46B
:2B306000020000000000000000000000000000002000000000000000040000000000000000000000000000004008EFE8
:2B308B00020000000000000000000000000000800300000000000060000000000000000000000000000000000688D6D1
:2B30B600020000000000000000000000000000000000000000000000000000000000000000000000000000000008EDF8
:2B30E100020000000000000000000000000000800100000000000000000000000000000000000000000000000088F4C5
:2B310C00000000000000000000000000000000200000000000000000000000000000000000000000000000000080C731
:2B313700000000000000000000000000000000C00100000000000000000000000000000000000000000000000000BEEE
:2B316200000000000000000000000000000000200000000000000000000000000000000000000000000000000080C7DB
:2B318D00000000000000000000000000000000A00301000000000000000000000000000000000000000000000000EC87
:2B31B800020000000000000000000000000000002000000000000000000000000000000000000000000000000080E763
:2B31E300020000000000000000000000000000800300000000000000000000000000000000000000000000000088D6DE
:2B320E00040000000000000000000000000000000000000000000000000000000000000000000000000000000008EB9E
:2B323900020000000000800100800100000000800100000000000000000060000000000000000000000060000088F4A9
:2B326400020000000000200000200000000000200000000000000000000008000000000000000000000008000008CDF8
:2B328F00020000000000C00100C00100000000C00100000000000000000070000000000000000000000070000000BC33
:2B32BA00000000000000200000200200000000200200000000000000000008200000000000000000000088000000E7EE
:2B32E500000000000000A01100A00300000000A00300000000000000000068000000000000000000000068000000DF18
:2B331000000000000000001000001000000000002000000000000000000000040000000000000000000000040080E5E5
:2B333B00020000000000800100800100000000800300000000000000000060000000000000000000000060000088D6C2
:2B336600020000000000000000000000000000000000000000000000000000000000000000000000000000000008ED45
:2B339100040000000000000000000000800100800100000000000000000000000060000600000600000600000090F217
:2B33BC00020000000000000000000000200000200000000000000000000000000008800000800000800000000008ED27
:2B33E700020000000000000000000000C00100C00100000000000000000000000070000700000700000700000008EDBD
:2B341200020000000000000000000000200000200000000000000000000000000088804000800000800000000088E994
:2B343D00000000000000000000000000A00101A08300000000000000000000000068800600800E0480460000000099C0
:2B346800000000000000000000000000001000002000000000000000000000000000048000004000004000000080E89D
:2B349300020000000000000000000000800100800300000000000000000000000060000E0000060000060000004083CB
:2B34BE000800008000008000008000008000008000080000000000200000200002200002200002200002200002B0FEDB
:2B34E900000000000000000000000000000000000000000000000000000000000000000000000000000000000080E751
:2B351400800008000008000008000008000008000000000000000000000200000000000000000000000000000080C59D
:2B353F00800008400008400008400008400008400004000000000010000210000110000110000110000110000180D4BA
:2B356A00000000000000000000020000220000008200040000000000200000008008000000000000000000008000C1A3
:2B359500000000000000000000000000000000000000040000000000000000000000000000000000000000000081F393
:2B35C000000000000000200000000000000000000000000000000000800000800000000000000008000000000000CFE9
:2B35EB00000000000000000000000080020000800000000000000000000000002000000200020000000200000080ED20
:2B361600000000000000200000020080200000008200040000000000A0000080A008000000020208000000008001D913
:2B364100000000400000000000000000000000000000000000000000400000000000000000000000000400000080A3B7
:2B366C00000000000000000000000000000000400008000000000000000000000000000000000000000000000000AF3C
:2B36970000000000000000000000000000000100C000000000000000000000000000000000000000000000000080FBCC
:2B36C200000000000000000000000000000000000000000000000000000000000000000000000000000000000080E776
:2B36ED00100000000000000000000000000000000000000000000000000000000010000000000002000000000080C64A
:2B371800000000000000000000000000000000000000000000000000000000080000000000000000100000000008F76F
:2B374300100000000000000000000000000000000000000000000000000000000000000000000000000000000080F7D4
:2B376E00000000000000000000000000000000000000000000000000000000000000000000000000000000000080E7C9
:2B3799000400000000000000000000000000000000000000000000000000000000000000000000000000000000C0A79A
:2B37C400000000000000000000000000000000000000000000000000000000000000000000000000000000000080E773
:2B37EF00000000000000000000000000000000000000000000000000000000000000000000000000000010000080F629
:2B381A00020000000000000000000000000000000001000000000000000000000000000000000000000000000080F50B
:2B384500000000000000000000000000000000000000000000000000000000000000000000000000000000000080E7F1
:2B387000000000000000000000000000000000000000000000000000000000000000000000000000000000000080E7C6
:2B389B002000922201000000000000000400000001001000000000000000000000000020000022000202000080048AC4
:2B38C600800009820000002200002208000000800008000000000000000080080080088800008080088000008280DFF7
:2B38F100000000000000000000000000000000000000000000000000000000000000000000000000000000000080E745
:2B391C00000000000000000000000000000000000000000000000000000000000000000000000000000000000080E719
:2B394700E0288EE3100AA1380A41388EA2108AE2108E0200000000288AA2108EA2280EE1100AE1288EE2288AE380982F
:2B3972006071976519DCC15DDC615816D71D5C7719161700000000705DD71D16D775976119DC6171177771DD6581FFEF
:02399D00FFFF2A
:00000001FF
